:020000040000FA
:1000000000306600F9306500A520A520851030304D
:100010008600A120A520A120A520A120A520203078
:100020008600A120A52020308600A120A5208030B8
:100030008600A120A52000308600A120A520E03068
:100040008600A120A52000308600A120A520103028
:100050008600A120A52000308600A120A5206030C8
:100060008600A120A520851420308600A120003024
:100070008600A120A52020308600A1200030860027
:10008000A120A52040308600A12050308600A1206C
:10009000A52040308600A12040308600A120A52068
:1000A00050308600A12050308600A120A52050307D
:1000B0008600A12000308600A120A52040308600C7
:1000C000A12090308600A120A52040308600A120EC
:1000D00030308600A120A5208510C0308600A120E8
:1000E00000308600A120A520851420308600A120A4
:1000F00000308600A120A52030308600A1201030DD
:100100008600A120A52030308600A1206030860026
:10011000A120A52040308600A12060308600A120CB
:10012000A52030308600A12080308600A120A520A7
:1001300030308600A12040308600A120A52000009C
:100140009F280515A52005110800FF308E008D00A1
:0A0150008D0BA8288E0BA7280800CD
:02400E00F93F78
:00000001FF
